:1000000010C028C027C049C125C024C023C022C0B9
:1000100021C020C01FC042C11DC01CC01BC01AC0CF
:1000200019C011241FBECFEDCDBF10E0A0E6B0E097
:10003000E8E1F3E002C005900D92A036B107D9F7D0
:1000400010E0A0E6B0E001C01D92A336B107E1F7D1
:1000500033D060C1D5CFA89584B7877F84BF88E1AE
:100060000FB6F89481BD11BC0FBE8AB388638ABBFA
:10007000B99AC09AD29A83B7846083BF87B187B98F
:1000800083E286B91C9A089A8BB780628BBF80B5D1
:10009000816080BD0895882321F4DD9A8BB3877E2B
:1000A00009C0813021F4DC9A8BB3877D03C0DB9AD1
:1000B0008BB38F7C8BBB0895AF92BF92CF92DF92B0
:1000C000EF92FF920F931F93CF93DF93C4DF789447
:1000D00085B7877E806185BF85B7806285BF88953B
:1000E00085B78F7D85BF82E090E020E80FB6F89459
:1000F00026BD86BD0FBE8BB78F7D8BBFC29A80E5B4
:1001000093EC0197F1F7B09B02C08FC0FFCFE1994C
:10011000FECF80E090E08EBBE09A8DB38095809317
:10012000600080916000B7DF1091600000E020E087
:10013000C0E5D3EC0FC02B3058F002C0243040F0A3
:100140001F5F133008F010E00F5F812FA4DF20E065
:1001500010936000B09977C0CE010197F1F72F5F3F
:10016000063048F3EBCFB299FECF8BB3877C8BBBC5
:10017000809160008230A9F420E004C0CE01019794
:10018000F1F72F5F809162002817C0F320E004C0D0
:10019000C6010197F1F72F5F809161002817C0F326
:1001A0002DC080916000813011F020E019C020E066
:1001B00004C0C8010197F1F72F5F809162002817F2
:1001C000C0F320E004C0CE010197F1F72F5F8091CA
:1001D00061002817C0F312C0C5010197F1F72F5F26
:1001E000809162002817C0F320E004C0C801019785
:1001F000F1F72F5F809161002817C0F3C19A8BB38C
:1002000088638BBB8CEA9DE0F7013197F1F701978A
:10021000D9F7C198809160003EDF80ED97E0F7014B
:100220003197F1F70197D9F79ECF88E028E130E0C8
:100230000FB6F894A89521BD0FBE81BD85B7877E06
:10024000806185BF63CF86B1806C86B9DA9A89B741
:10025000816089BF22E3E22EF12C04EC10E0C3E1BF
:10026000D0E098EAA92E97E0B92E81E0C82ED12CD3
:100270007ACFB09B02C080E008958FEF089588E0A8
:1002800028E130E00FB6F894A89521BD0FBE81BDDE
:1002900085B7877E806185BFFFCF18951F920F922B
:1002A0000FB60F9211242F938F939F9387B18823BA
:1002B00031F485B18093610081E087B904C085B1D4
:1002C0008093620017B8B0991DC020916000E19939
:1002D000FECF1CBA80E090E08EBB20952DBB0FB600
:1002E000F894E29AE19A0FBE28E088E190E00FB618
:1002F000F894A89581BD0FBE21BD85B7877E80612A
:1003000085BFFFCF9F918F912F910F900FBE0F90C0
:080310001F901895F894FFCF2F
:00000001FF
